:101800001AC132C131C130C12FC12EC12DC13CC25C
:101810002BC12AC129C128C127C126C125C124C184
:1018200023C122C1FEC120C1B9C11EC11DC11CC13D
:101830001BC11AC119C1000021104220633084402D
:10184000A550C660E770088129914AA16BB18CC18F
:10185000ADD1CEE1EFF13112100273325222B55206
:101860009442F772D662399318837BB35AA3BDD3DF
:101870009CC3FFF3DEE36224433420040114E664D6
:10188000C774A44485546AA54BB528850995EEE52F
:10189000CFF5ACC58DD55336722611163006D776E6
:1018A000F6669556B4465BB77AA719973887DFF77F
:1018B000FEE79DD7BCC7C448E5588668A7784008AE
:1018C000611802282338CCC9EDD98EE9AFF94889CF
:1018D00069990AA92BB9F55AD44AB77A966A711A46
:1018E000500A333A122AFDDBDCCBBFFB9EEB799B1F
:1018F000588B3BBB1AABA66C877CE44CC55C222C96
:10190000033C600C411CAEED8FFDECCDCDDD2AAD6E
:101910000BBD688D499D977EB66ED55EF44E133E25
:10192000322E511E700E9FFFBEEFDDDFFCCF1BBFBE
:101930003AAF599F788F8891A981CAB1EBA10CD198
:101940002DC14EF16FE18010A100C230E3200450A0
:10195000254046706760B9839893FBA3DAB33DC313
:101960001CD37FE35EF3B1029012F322D2323542F0
:10197000145277625672EAB5CBA5A89589856EF5A3
:101980004FE52CD50DC5E234C324A0148104667440
:10199000476424540544DBA7FAB79987B8975FE7F3
:1019A0007EF71DC73CD7D326F2369106B016576690
:1019B0007676154634564CD96DC90EF92FE9C8997B
:1019C000E9898AB9ABA94458654806782768C018E0
:1019D000E1088238A3287DCB5CDB3FEB1EFBF98B53
:1019E000D89BBBAB9ABB754A545A376A167AF10A30
:1019F000D01AB32A923A2EFD0FED6CDD4DCDAABD63
:101A00008BADE89DC98D267C076C645C454CA23C7F
:101A1000832CE01CC10C1FEF3EFF5DCF7CDF9BAF32
:101A2000BABFD98FF89F176E367E554E745E932ECF
:101A3000B23ED10EF01E11241FBECFEFD4E0DEBFA8
:101A4000CDBF14BE88E10FB6F89480936000109269
:101A500060000FBE21E0A0E0B1E001C01D92A13AFC
:101A6000B207E1F740D276C2CBCE81E085BF82E0FB
:101A700085BF089581E085BF15BE08957F928F923E
:101A80009F92AF92BF92CF92DF92EF92FF920F930D
:101A90001F93CF93DF93CDB7DEB7DA950FB6F894E7
:101AA000DEBF0FBECDBF7E0181ECE80EF11C8E01C2
:101AB0000F5F1F4FCC24DD24C01AD10A712C5701AF
:101AC0004701D801FD01EC0DFD1DE491ED93A81532
:101AD000B905C1F7FFE17F1207C06EEBC801DDD188
:101AE000F50197AF86AF06C060ECC801D6D1F7010B
:101AF000918380837394F2E0EF0EF11C80ECC80EAA
:101B0000D11CE0E27E12DDCF60E4C501C6D1D395E1
:101B10000FB6F894DEBF0FBECDBFDF91CF911F91FE
:101B20000F91FF90EF90DF90CF90BF90AF909F907C
:101B30008F907F900895E1EBF0E010821092B20058
:101B40008AE38093B30083E0808382E08093700017
:101B500081E080939D01089561157105F1F0409138
:101B600005015091060120910301309104014217B3
:101B7000530709F0FFCF5A9A9C012F5F3F4F3093D4
:101B8000060120930501680F791F7093040160938B
:101B90000301FC0180818093C60008951F920F927B
:101BA0000FB60F9211242F938F939F93EF93FF9370
:101BB000E0910501F09106018091030190910401EB
:101BC000E817F907C1F4109207015A988091C100F3
:101BD00080688093C100809102018823C1F028E0D1
:101BE00088E190E00FB6F894A895809360000FBE4E
:101BF00020936000FFCF80818093C6008091050113
:101C00009091060101969093060180930501FF9142
:101C1000EF919F918F912F910F900FBE0F901F907A
:101C200018951F920F920FB60F9211248F939F93C6
:101C3000EF93FF93809107018D3810F01092070108
:101C4000809107019091C600E82FF0E0E85FFE4F19
:101C500090838F5F809307011092B1001092B200C1
:101C60008AE28093B30083E08093B10082E08093A6
:101C7000700010929D01FF91EF919F918F910F90B5
:101C80000FBE0F901F9018951F920F920FB60F92D4
:101C900011242F933F934F935F936F937F938F9371
:101CA0009F93AF93BF93CF93DF93EF93FF93809175
:101CB0009D01811191C01092B1001092B20082E09A
:101CC00087BB8091C1008F778093C10034DF609122
:101CD00007016D3008F4ACC0862F90E0885F9E4FFE
:101CE000FC013197C081D0E0DC2FCC273197808177
:101CF000C80FD11D625088E091E0CFD08C179D07AE
:101D000009F096C0C09108018C2F807F803A09F0BD
:101D10008FC049E050E069E071E080EF90E00DD1C4
:101D2000892B09F085C08C2F8F70863021F481E0DB
:101D30008093020105C0843029F481E08093A001E2
:101D400084E05CC0853091F507B600FC54C08091FA
:101D500007018E3209F051C020911301203C08F098
:101D60004CC080E2289F90011124A6E1B1E060916F
:101D7000140171E0A90146515140FA01EA0FFB1F1D
:101D8000ED012197888190E0982F8827860F911D7B
:101D90000C0170935700E89511246C911296E1E0C4
:101DA000A633BE0751F785E0F90112C0873029F547
:101DB00007B600FC20C0809107018E30F1F4E0915D
:101DC0001301E03CD0F480E2E89FF001112483E0AD
:101DD00080935700E895B4CF8130C1F51092B100DF
:101DE0001092B20082E087BB6091070170E088E04A
:101DF00091E0B2DE2BC085E001C082E0806D80936F
:101E0000080189E0E0EFF0E0A9E0B1E001900D9277
:101E10008A95E1F7109212016BE088E091E03DD0E5
:101E200080931301909314018DE0809307010EC0FD
:101E3000109207015A988091C10080688093C10078
:101E40001092B1001092B20082E087BBFF91EF9137
:101E5000DF91CF91BF91AF919F918F917F916F91C2
:101E60005F914F913F912F910F900FBE0F901F9058
:101E70001895529A5A98589AF8941092C5008CE086
:101E80008093C40082E08093C00088ED8093C100FD
:101E900086E08093C20078940895DC01762F6A0F63
:101EA0008FEF982F40E026E338E150E04D9149272D
:101EB000440F551FF901E40FF51F082E85919491E9
:101EC00090256A1791F708955C9A5B9A709A813011
:101ED00021F0823019F4709808955B980895549A0F
:101EE000539A689A0895C1DDC4DFF9DF82E0ECDF20
:101EF000C5DDEEEFF7E1259134912817390721F080
:101F000081E08093A001E0DF2FE788E391E021509A
:101F100080409040E1F700C000008091A001811155
:101F2000FFCFF89480E0D0DFA5DDE0910001F091D3
:101F30000101099580E090E00895FB01DC0104C0F7
:101F40008D910190801921F441505040C8F7881BB1
:081F5000990B0895F894FFCFEE
:0400000300001800E1
:00000001FF
